:030000000219FDE5
:03000B000200A848
:03002B000201616E
:03005B000202F2AC
:030073000202DFA7
:1000800002030406080C10182030406080040608A3
:100090000C10182030406080A0C00003070F1F051F
:1000A000050D050305030302C2AFC0D0C0E0206206
:1000B00014E5256009E473E525F4F58AD262D0E001
:1000C000D0D0D2AF3285268AC262E526F4603630BF
:1000D000682C20720DD0E0D0D0C283C294C295D2D9
:1000E000AF32C283C294C295206F13206510740C86
:1000F000D5E0FDE57BB48004429001FE4280D0E073
:10010000D0D0D2AF32758A00C28DD26201FE01B763
:10011000306805206502D28301B73068052065028A
:10012000D29401B7306805206502D29501B7C2802C
:1001300030680A2065077408D5E0FDD28301B7C294
:100140008230680A2065077408D5E0FDD29401B7B3
:10015000C29730680A2065077408D5E0FDD2950182
:10016000B7C2AFC2AD53E6EFC0D0C0E0D2D3D2AF7A
:10017000C2CEE52A600720744F152A21C87800797D
:100180000020742EE580307E01F430E50278FF53C4
:10019000DACF207E0343DA20307E0343DA10C2D860
:1001A000C271E580307E01F430E50279FFC3E89941
:1001B00070CB306103752A18207403752A18885C87
:1001C000D270E86003755F0020740DE52B600415A4
:1001D0002B21D843DA01C2D8207002414BA85C2001
:1001E0006102C270207431C3E894F0400374F0F8E7
:1001F000E8C4540F28F87984B703024118C313C325
:10020000138721200802C313200A06C3C898F841A7
:100210001828F8500374FFF8C3E895655003E565A6
:10022000F88822E52D54066022206B1FE536C33383
:10023000C333F8E564C313C313F9C395224002899D
:1002400022E82522F52250037522FF852224A824C6
:10025000C3E52495614002A8618825E566700241E6
:100260008FC3E8AA669A5003E8FAE4F9EAC333FBBD
:10027000E568F45B29400D2567F8E56760021567BE
:10028000400B418F0AC3E5679A5002056778FF88E3
:1002900026C26FC3E52694F84002D26F20CF0AD061
:1002A000E0D0D043E610D2AD32C2CF053A7801E5B6
:1002B0002A6005307402152AC3E55C940140057577
:1002C0005F0041D5756000756900E55F2401F55F49
:1002D0005003755FFFD0E0D0D043E610D2AD32C2FC
:1002E000AF53E67F7592FA7593FFC260759104D2A1
:1002F000AF32C2AF53E6EFC2ADC0D0C0E0C0F0D263
:10030000D3D2AFA8FBA9FCC2D8307102615953DA2D
:10031000CF207E0343DA10307E0343DA20D271E52A
:1003200080307E01F420E502613088278928A1868B
:1003300053DACF207E0343DA20307E0343DA10C243
:10034000D8C271307402A1727800E580307E01F469
:1003500030E502A172885CA15A53DACF207E0343B4
:10036000DA20307E0343DA10C271206102813253F9
:10037000DACF207E0343DA10307E0343DA20C2D87E
:10038000D27188578958C3E89555F8E99556F97B95
:10039000007E087A00C3E8948CE994005005755BF0
:1003A000008124882178A2E6A8216055C3E894C87A
:1003B000E994005008E4D2E4FB7A0A61FFC3E894B0
:1003C00068E994015008E4D2E3FB7A0F61FFC3E8C7
:1003D00094D0E994025008E4D2E2FB7A1E61FFC394
:1003E000E894A0E994055008E4D2E1FB7A3C61FF6F
:1003F000C3E89498E994085008E4D2E0FB7A787E48
:1004000000C3E89559FCE9955AFD30E70AECF4245D
:1004100001FCEDF43400FD755B00C3EC9AED9E50D9
:1004200003755B018859895A855755855856780256
:10043000A15AC3E89527F8E99528F9307C02A13E36
:10044000307B02A13E307A02A1372075028155E946
:10045000FDE8FC8174E9C313F9E813F8307902A1CF
:1004600037E9C313F9E813F8307802A137E9C31369
:0E047000FDE813FC20612CC3EC941CED9402FB
:10047E004002818BED701EC3EC94C850180529E51F
:10048E002970021529C3E529940A5002A172755CE0
:10049E0000D270A172E529600215297888E6F974F8
:1004AE0000207F087896B90302789EE624FAFEE4CF
:1004BE003400FFC3EC9EFCED9FFD9208B90310A221
:1004CE00085007207609D27681DD307602C276A2F8
:1004DE00085016B9030DECF42401FCEDF43400FDC4
:1004EE000204F778007900A13EB90315EC33FCED58
:1004FE0033FDC3EC940AFCED9400FD50047C007DAA
:10050E0000C3EC94FFED9400400678FF7900A13E05
:10051E00EC8572F0A4C5F0A2F733F879004003021F
:10052E00055A78FF790002055AE9C313F9E813F862
:10053E00307C0EE9600278FFC3E81338F8E434002B
:10054E00F9C3E894FFE99400400278FF885CD2700A
:10055E00206102A172741FF4552F4BF52FC274EB5C
:10056E007002D274752A18307403752A0A3061022B
:10057E00A18620740353DAFE207403752B06D0F087
:10058E00D0E0D0D0D2AD43E6103279010205B67973
:10059E00030205B6790A0205B6791E0205B679641C
:1005AE000205B679C80205B67817E4D5E0FDD8FA8B
:1005BE00D9F6227A147B780205DD7A107B8C02053F
:1005CE00DD7A0D7BB40205DD7A0B7BC80205DDE515
:1005DE0073D5E001227902E4C282D5E0FDD294D532
:1005EE00E0FDC294D5E0FDD282D5E0FDE920E00227
:1005FE00D28330E002D295E573D5E0FDE920E0022A
:10060E00C28330E002C2957496D5E0FDD9C9EAF8EE
:10061E00D5E0FDD8FBDBB8C28222C37C007D00751D
:10062E00F00005F0EA33FAEB33FB50F6EB13FBEA7E
:10063E0013FAC3E9FFE8FEE89AF8E99BF95004EFD4
:10064E00F9EEF8B3EC33FCED33FDD5F0DFEDF9EC5C
:10065E00F822E889F08A20D2D4F8A9F07B0030F78E
:10066E000B7BFFF42401F8E9F43400F9E88520F05F
:10067E00A4ADF0F8E98520F0A4AFF0FEED2EF974EC
:10068E00003FFA7C04C3EA13FAE913F9E813F8DC25
:10069E00F48BF030F70AE8F42401F8E9F43400F9A9
:1006AE00E889F0C2D4F8A9F02222C3E54113F9E596
:1006BE004013F8C3E54498F8E54599F9500CC3E8A2
:1006CE009480E994FF40160206EFC3E8947FE99404
:1006DE000050030206EF787F79000206EF788079EA
:1006EE00FF8849894A22E5492546F8E54A3547F902
:1006FE00854A20E4300701F43548FA30E709C3EAA9
:10070E0094F0401502072DC3EA940F500302072DF3
:10071E0078FF79FF7A0F02072D780079007AF0C3FF
:10072E00E5249561500AC374019524500B02074BC2
:10073E00E54A20E70E02074BE54A30E70688468970
:10074E00478A482278A5E6FAC3E54933F8E54A33E5
:10075E00F9D160E930E70BC3E89480E994FF4013C8
:10076E00E185C3E8947FE994005002E185787F79B2
:10077E0000E185788079FFE820E715C3E52398F836
:10078E004009C3E8940140030207AC78010207ACAC
:10079E00E8F424012523F840030207AC78FF884BC8
:1007AE002278A6E6FAA847A948D160E930E70CC33B
:1007BE00E89401E994FF40160207E0C3E894FFE9CC
:1007CE00940050030207E078FF79000207E07801F9
:1007DE0079FFE920E715C3E54B98F84009C3E89483
:1007EE000140030208077801020807E8F4240125F6
:1007FE004BF8400302080778FF88242278FF20690F
:10080E002879A1E76023E541601F74FF8541F084DC
:10081E008539F0306A0375F005A4F8C5F0600278EA
:10082E00FFC3E895645002A864886322C3E5409430
:10083E0040E5419401E563500314014B046002F559
:10084E0063220208532275E890227883E6FF30ED8A
:10085E00F9A8BDA9BE0570C3E57094084052757025
:0F086E0000E9FA79A0E76044EA7007E571601BC2
:10087D0002088CC3E895716010E5715006600C1488
:10088D000208980460F9020898E571F571C3946D3A
:10089D00401B7561C0C394044013756180C39404FB
:1008AD00400B756140C39404400375610075BB092D
:1008BD0022E561F460020561E570B4070375BB10B4
:1008CD0022743279A787F0A4C5F0A2F733F8C3E8F4
:1008DD0095614002A861882288248825882688642D
:1008ED00227540007541F022C2AF75C820A8CCA971
:1008FD00CDAA3A30CF010A75C824D2AFAB3BAC3C80
:10090D00883B893CC3E89BF8E99C206908F930666F
:10091D000241062160AD3D8A3DF9EA9DFA600678F7
:10092D00FF79FF2145AE3EAF3F8B3E8C3FA83BA9E3
:10093D003CC3E89EF8E99FF9C3E54113FBE540137D
:10094D00FAE82AF540E93BF54150067540FF75413F
:10095D00FF21ADAA40AB41AC40AD417E047F02C347
:10096D00EB9404400D1E1FC3EB94084005206A0252
:10097D001E1FC3ED13FDEC13FCDEF7C3EA9CFAEB6F
:10098D009DFBEF6009C3E913F9E813F8DFF7EA28D7
:10099D00FAEB39FB8A408B4150067BFF8B408B4134
:1009AD00C3EB94025002D2663069047F0321D878DC
:1009BD0092E6FFC3E537948240110FC3E53794A04B
:1009CD0040010FC3EF940640027F057E02E541C44E
:1009DD00540FF9E541C454F0F8E540C4540F28F81C
:1009ED00C3E89EFAE99400FB4009C3EA9402EB9434
:1009FD000050047A02E4FB4152AA40AB41EBC4FE25
:100A0D00EAC4540F4EFCC3EA9CFAEB9400FBC3E816
:100A1D0013C313F8EA28FAEB3400FB8A408B41C369
:100A2D00EB94024002C2667802EBC4FE7B00EAC47E
:100A3D00540F4EFAC3EA98FA4005C3940250027A55
:100A4D00027892E6FF3060024152855192855293B1
:100A5D00D26043E680C3E49AF8E49BF93066024124
:100A6D00DEE8FAE9FBD3E913FDE813FC885189525E
:100A7D00C3EF94036038EF20E00DE82CF8E93DF961
:100A8D00ECFAEDFB020AA7E828F8E939F9C3E824E6
:100A9D0002F8E93400F97AFE7BFFC3EF9403400EB0
:100AAD008A538B54884D894E8C4F8D5061128853CB
:100ABD0089548A4D8B4E8C4F8D503069127553F081
:100ACD007554FF754FF07550FF7551F07552FF61FC
:100ADD0012E8FAD3E813FC8851C3EF94036020EFBA
:100AED0020E007E82CF8ECFA41FEE8282402F87A19
:100AFD00FEC3EF940340088A53884D8C4F611288D2
:100B0D00538A4D8C4FE568C3335002646BF56830E2
:100B1D006002611C753402D26043E680E52D5406F7
:100B2D006034A840A941C3E913F9E813F8C3E913E8
:100B3D00F9E813F8306904E92440F9C2AF53E67FB0
:100B4D00759100C3E498F594E499F595759104D2E7
:100B5D006043E680D2AF22D2647543007520003029
:100B6D006C03752040020B83D264754300752040E1
:100B7D00306C0375200078017901206620E52D5435
:100B8D00066002C2647914E541C313700104F8C311
:100B9D00941440027814306904781B791B2060107E
:100BAD00E543600C306903D53404D26D812E712478
:100BBD000543E59BF45440B52002811830690908BE
:100BCD00C3E89940011861AA20640A08C3E8994056
:100BDD0002618361AAC264C2AF53E67F7591003092
:100BED0066127594007595F8759104D26043E68090
:100BFD00D2AF6183E5417EFFC3334005C33340016E
:100C0D00FEC3E49E759400F59561F5C3E53394013B
:100C1D00500261833064026183D802812C61AAC2C3
:100C2D006DC2AF53E67F75910085539485549575CC
:100C3D009104854D92854E93D26043E680D2AFE507
:100C4D002D54066008206A020533020C6A306D0DC2
:100C5D00206C0A2064071581158102153622780053
:0F0C6D003064027801E53775F007A4F9E5F02847
:100C7C00F5F0E9A2F013A2F113A2F213F537C39425
:100C8C00785003753778C3E53795384008D265C27C
:100C9C0083C294C29530600281A1854F9285509396
:100CAC00D26043E68022207D16C2AF754202C2821A
:100CBC00D280306202D295D2AF759F43020EA2C28F
:100CCC00AF754202C282D297306202D283D2AF7524
:100CDC009F43020EA2307243207D20C2AF754203A7
:100CEC0090013F757B04C295C297306204D2948107
:100CFC00FFD282D2AF759F53020EA2C2AF754203D0
:100D0C0090013F757B04C283C280306204D294A1EF
:100D1C001FD282D2AF759F33020EA2207D17C2AFB5
:100D2C0075420390011AC295306202D294D2AF750B
:100D3C009F53020EA2C2AF75420390011AC28330B8
:100D4C006202D294D2AF759F33020EA2207D16C2DE
:100D5C00AF754204C280D297306202D294D2AF7582
:100D6C009F33020EA2C2AF754204C297D28030628A
:100D7C0002D294D2AF759F53020EA2307243207DE3
:100D8C0020C2AF75420590012E757B01C294C282C0
:100D9C00306204D283A1A5D280D2AF759F43020EDC
:100DAC00A2C2AF754205900150757B80C294C2827D
:100DBC00306204D295A1C5D297D2AF759F43020E73
:100DCC00A2207D17C2AF754205900110C29430620B
:100DDC0002D283D2AF759F43020EA2C2AF754205F9
:100DEC00900124C2943062EBD295D2AF759F43022E
:100DFC000EA2207D16C2AF754206C297D282306217
:100E0C0002D283D2AF759F53020EA2C2AF754206B7
:100E1C00C280D282306202D295D2AF759F33020E5D
:100E2C00A2307244207D20C2AF75420190015075F2
:100E3C007B80C283C280306204D295C14BD297D2E0
:100E4C00AF759F33020EA2C2AF75420190012E7591
:100E5C007B01C295C297306205D283020E6CD280A0
:100E6C00D2AF759F53020EA2207D17C2AF754201FF
:100E7C00900124C283306202D295D2AF759F3302A7
:100E8C000EA2C2AF754201900110C295306202D21F
:100E9C0083D2AF759F53C2652290010E757B00C241
:100EAC0083C294C295C280C282C297C262227880E9
:100EBC0076FF0876FF0876FF0876FF08760308763B
:100ECC0004087609087603087601087601788C7692
:100EDC00010876FF0876FF0876FF0876FF0876FF94
:100EEC000876030876FF0876FF0876FF0876250853
:100EFC0076D00876FA0876FA0876040876FF087633
:100F0C000108760008767A0876FF087601087601E3
:100F1C00087600087603087600227887E6FFC2720E
:100F2C00BF0302D2727888E6C394036008C27DE6E0
:100F3C0030E102D27DC27E7889E630E102D27EC3F6
:100F4C00EF94026008758E01D273020F5E758E00ED
:100F5C00C273227880E6149000809378A5F678818D
:100F6C00E6149000809378A6F67886E61490008DAF
:100F7C009378A7F67886E6F539C394025003753951
:100F8C0002789CE67538FFB402037538A0B40303ED
:100F9C0075388278A3E61490009A93F566D1A52251
:100FAC00227896E6FA7897E6FB7888E6B40305C3D0
:100FBC00EB940EFB307F047A007BFFC3EB9AFCC3EF
:100FCC00948250027C827572000572EC8572F0A4DA
:100FDC00C3E5F0947D40F222D27FF1AD1205A71249
:100FEC0005A77A007B007C1012059DE55C2AFA743B
:100FFC00003BFBDCF37C04C3EB13FBEA13FADCF7DA
:10100C00FEC27F120FAD22757C00757D00E5EF20CE
:10101C00E6037520000520903FFFE5201460069044
:10102C001DFF1460009304600375EF1653D9BF7550
:10103C0081C043FF8012059875EF0643B203E5B3F8
:10104C00240220E70DF521E5E320E0068521B343DA
:10105C00E301120EA57580F275A40D75F13F75D4E0
:0D106C00DF75904F75A5B075F2F075D500D9
:1010790075A60175E241120EA5E4F8F6D8FD75686A
:1010890001120EBA12158778988673753001C2AFAE
:101099001205B11205C11205A71205C81205A7123A
:1010A90005CF1205A71216B01205B11205B1120526
:1010B900ACC2AF757C00757D0078FA79FA30850786
:1010C900D9FBD8F7021C00120F26120F5F120FACC2
:1010D900120FAD78988673120EA57588107589025E
:1010E90075C82475910475D84075A82275B802751C
:1010F900E690759B80759D0075D10E75BC5875BBC2
:101109000975BA1175E880120598D2AF12085075A1
:10111900360053DACF207E0343DA20307E0343DAE8
:101129001043DA01C2D8C2711205B1D2617B037AC8
:101139000CE55B70077A0CDB030210BA1205A720D5
:1011490070030210BAC270E55CC3940240E1E52F56
:10115900541F855E5DF55EB55DD5DAD5C26153DA9A
:10116900CF207E0343DA20307E0343DA10C2D8C28F
:101179007178A2E67008D274E52F54E0F52FC27594
:101189007529001205AC307409C3E529940A400297
:10119900D27512059D78023074027800C3E55C9817
:1011A90040F0C2AF1205C11205C11205C1D2AF127A
:1011B90005B1754C007888E6B4030241BA12059D61
:1011C900788CE6C3940150030212BAE530C3940146
:1011D90050030212BA757CA5757DF1207435C3E5FB
:1011E9005C94FF50030212BAC2AF1205D6D2AF12F5
:1011F90005ACC3E55C940150EFC2AF1205C11205FD
:10120900A21205C1D2AF1205ACC3E55C94FF40E957
:101219000217357F05D27F120FAD1205ACC2AFC2DE
:101229007F120FADAE5CC3E55C947FD2AF50024133
:10123900CA120598C2AF1205D6D2AFDFD8120FE491
:10124900C3EE94057897F61205B11216B87F0AD243
:101259007F120FAD1205ACC2AFC27F120FADAE5CEB
:10126900C3E55C947FD2AF50E4120598C2AF120572
:10127900C11205A21205C1D2AFDFD4120FE4EE24C8
:10128900037896F6F87997E7C39482400398500655
:10129900E824827897F61205B11215D51216E712CD
:1012A90005AC120FADC3E55C94FF500221DE0217B5
:1012B90035757C00757D00C3E55C954C4003855C04
:1012C9004C1205AC78017988E7B403027805C3E5C7
:1012D9005C98400221BEC2AF1205D61205D612058E
:1012E900D6D2AF1205B1753000E4F531F5320531CA
:1012F900E531F4703F0532789AE67819146012786E
:101309003214600D787D14600878FA146003753220
:1013190000C3E53298401D120EA5120598153275C5
:10132900310078998673C2AF1205D6D2AF78988604
:10133900731205AC1205A2E52A700530740201BAD0
:1013490078012074027806C3E55C9840A17888E6A4
:10135900C3940360031205ACE52A70030210BAC2F4
:10136900AF120EA5E4F522F523F524F525F526F5AA
:1013790067D2AF7885E6C333F565E4F544F545F5FD
:1013890046F547F548F570F52CF52DF537757008D4
:1013990075BB1012059812085430EDFDA8BDA9BE01
:1013A900E97001F8887112085875700875BB101238
:1013B9000F26C2AF7561FF1208CE852261852262B0
:1013C900852263D2AF752201752401752501752621
:1013D90001856069756A017888E6B40307C27D30C2
:1013E9007602D27DD268D269753300120DFE120ED3
:1013F9002D1208EE1208F51208EE1208F51208EE81
:10140900120B751206B7120C6B120CB21208F512F8
:101419000B64306E031206B820660312080A3066A0
:101429000312083A120C6B120CE11208F5120B7533
:10143900306E031206F4120C6B120D581208F512D5
:101449000B64306E03120752120C6B120D871208CF
:10145900F5120B75306E031207AF120C6B120DFEED
:0F1469001208F5120854120B64120C6B120E2DA0
:101478001208581208F530692F8564618564628501
:101488006069756A0179187A0CC3E53399400CC212
:1014980069D26A8A357561FF0214B0C3E55C9401AC
:1014A800400302140902153E306A25206C22E535F6
:1014B800147006C26AD26B8109F535C3E55C9401E4
:1014C80040030214097888E6C39403600302153EBA
:1014D800753600788279A4E760027803C3E55F98DF
:1014E8005054307404E52A604D7888E6B403172018
:1014F8007D05207607A10E307602A10E206C07D25A
:101508006C856461814878F0306C05856461782069
:10151800C3E5419850028109306C1BC26CC27D3012
:101528007602D27DD26A75351285646181090536E5
:10153800E55C6002A141753600C2AF120EA578873E
:10154800E6FE7602120F267887EEF6E4F522F523FA
:10155800F524F525F526F565752C00752D00D2AF17
:101568001205AC120EA578A4E66006D283D294D2F6
:1015780095307409C3E5369404400201BA41F290EB
:101588001A0D7820121617E520B45A0CA312161754
:10159800E520B4A5030215B5757CA5757DF1120E7D
:1015A800BA1215D5757C00757D000215D4901A0302
:1015B80078807B0A121617A308DBF9901A0F788C2B
:1015C8007B19121617A308DBF9901A2822C2AF124A
:1015D800165A121637901A00740E12161CA37409A4
:1015E80012161CA3741512161C901A0378807B0A15
:1015F80012161BA308DBF9901A0F788C7B191216A8
:101608001BA308DBF912166D12164B901A2822E458
:1016180093F622E6438F01538FFDFFC3E583941CA5
:10162800400122EF857CB7857DB7F0538FFE2243BA
:101638008F02438F01857CB7857DB7901A0DF053D3
:101648008FFC22901A0D745AD11C901A0E74A5D1D1
:101658001C227A3079D07820901A40D117E520F7EB
:1016680009A3DAF7227A3079D0901A40E7D11C0919
:10167800A3DAF922AB74A875BB01027984BB020214
:101688007985BB03027986BB04027992BB0502798E
:1016980087BB060279A3BB0702799CBB080279883D
:1016A800BB09027989E8F7227C051205B1DCFB2227
:1016B800C2AF1205C11205C81205CF1205D6120510
:1016C800A21205C11205C81205CF1205D61205A22D
:1016D8001205C11205C81205CF1205D6D2AF22C213
:1016E800AF1205D61205CF1205C81205C11205A200
:1016F8001205D61205CF1205C81205C11205A2128D
:1017080005D61205CF1205C81205C1D2AF22AE7494
:10171800AF75C2AF1205C11205C11205C11205A2EB
:10172800DEF21205D61205A2DFF8D2AF22D1B8D167
:10173800B0D1B0757401757501757600F1167C0528
:10174800AD5C1205B1C3ED955C70F5C3E55C940121
:10175800400AC3E55C94FF4032021771D17CB1D5D1
:10176800D1B8C2AF75EF16D1B0DCD50576C3E57632
:101778009403500280C6D1B00575E5741490009F9B
:1017880093F808C3E57598500280AED1B0D1B00582
:1017980074C3E574940A5002809C120EBAB1D5C283
:0617A800AF75EF16D1B091
:0319FD00021013C2
:101A00000E0915FFFFFFFF0304090301015AA50199
:101A1000FFFFFFFFFF03FFFFFF25D0FAFA04FF01DE
:091A2000007AFF0101000300FF40
:101A400023416C69676E424C333558232020202097
:101A500023424C48454C4923463333302320202031
:101A60002020202020202020202020202020202076
:101C0000C2AFC2D353D9BF7581C043B20343FF8073
:101C1000752438752503B1DC7529A5752AF175E29F
:101C20004043F12053A4DF75D4FFD2857DFA7803B9
:101C300079E67C10752200752300901DE97B0675FE
:101C400024987525013085028145208508D8FBD967
:101C5000F9DCF781B7308508D8FBD9F9DCF781B713
:101C6000B19CE493A3C39A6004DDC381B7DBDBB10D
:101C70008E6002812E7B08E493FAA3B16FDBF87AC1
:101C800030B16F752200752300B18EEAFCEBFDC305
:101C9000ED94FE400EB18E8A278B28ED30E0048A49
:101CA000828B83B18E7AC270D8C3ED94FE601950D6
:101CB000CEBD002BEC600F7520007521FF7529004B
:101CC000752A000200008100A827A9280809D80465
:101CD000D90281DCB192EA89AAF281CE0D81A3C337
:101CE000ED94035053EDA2E092007AC5C3E58294CF
:101CF00000E583941C508A200010438F02438F011B
:101D00008529B7852AB7F0300029A827A92808090E
:101D1000438F01538FFDD804D902A133C3E58394C7
:101D20001C4003A3A11689AAE28529B7852AB7F02A
:101D3000A3A116538FFC817F7AC1BD030CE493A34A
:101D4000FAB153DCF8B14B817F8181AA22AB23B178
:101D50006FEBFAEA6222752608C3E52313F523E543
:101D60002213F52250066323A0632201D526EAB18F
:101D7000DCB1DC75260AEAF4200102D285300102CA
:101D8000C285B1DCC3134002C201D526EB22B19259
:101D9000EAFB208502A192308502A197752608AE44
:101DA00024AF25C3EF13FFEE13FEB1E0B1DCC3EAAD
:101DB000133085024480FA30E703632201C3E52330
:101DC00013F523E52213F52250066323A0632201B5
:101DD000D526D9E52265236523F52222AE24AF2539
:101DE0000E0FDEFEDFFCD20122424C48656C6934E6
:071DF000373164F3300601F6
:00000001FF
